S01A000064656D6F70726F675F73746D3332663734362E737265638E
S31508008000080500202DA1000875A1000879A100081F
S315080080107DA1000881A1000885A1000800000000D4
S3150800802000000000000000000000000089A1000810
S315080080308DA100080000000091A10008039A00081D
S3150800804095A1000899A100089DA10008A1A1000812
S31508008050A5A10008A9A10008ADA10008B1A10008C2
S31508008060B5A10008B9A10008BDA10008C1A1000872
S31508008070C5A10008C9A10008CDA10008D1A1000822
S31508008080D5A10008D9A10008DDA10008E1A10008D2
S31508008090E5A10008E9A10008EDA10008F1A1000882
S315080080A0F5A10008F9A10008FDA1000801A2000831
S315080080B005A2000809A200080DA2000811A20008DE
S315080080C015A2000819A200081DA2000821A200088E
S315080080D025A2000829A200082DA2000831A200083E
S315080080E035A2000839A200083DA2000841A20008EE
S315080080F045A2000849A200084DA2000851A200089E
S3150800810055A2000859A200085DA2000861A200084D
S3150800811065A2000869A200086DA2000871A20008FD
S3150800812075A2000879A200087DA2000881A20008AD
S3150800813085A2000889A200088DA2000891A200085D
S3150800814095A2000899A200089DA20008A1A200080D
S31508008150A5A20008A9A20008ADA20008B1A20008BD
S31508008160B5A20008B9A20008BDA20008C1A200086D
S31508008170C5A20008C9A20008CDA200080000000098
S31508008180D1A20008D5A20008D9A20008DDA20008DD
S31508008190E1A20008E5A20008E9A20008EDA200088D
S315080081A0F1A20008F5A20008F9A20008FDA200083D
S315080081B001A3000805A3000809A300080DA30008E9
S315080081C011A3000815A30008EE11AA5510B504005E
S315080081D0002C01D1012035E0A0690028FFD1606F8D
S315080081E0002805D1002084F87000200000F047FB25
S315080081F024206067206800684008400021680860FD
S31508008200200000F0B1F8012801D101201AE0606AC7
S31508008210002802D0200000F06FFA2068406830F489
S315080082209040216848602068806830F02A002168FC
S3150800823088602068006850F0010021680860200006
S3150800824000F0C7FA10BD2DE9F84306000D0014002A
S315080082501F00B06F202840F08480002D03D0200036
S3150800826080B2002801D101207CE096F87000012830
S3150800827001D1022076E0012086F870000020F06720
S315080082802220B06700F0FCFA8046A6F85840A6F807
S315080082905A40B068B0F5805F0BD13069002804D128
S315080082A040F2FF10A6F85C0023E0FF20A6F85C0069
S315080082B01FE0B06800280AD13069002803D1FF20E2
S315080082C0A6F85C0015E07F20A6F85C0011E0B0680F
S315080082D0B0F1805F0AD13069002803D17F20A6F863
S315080082E05C0006E03F20A6F85C0002E00020A6F845
S315080082F05C00B6F85C90B068B0F5805F04D1306970
S31508008300002801D1002416E02C00002513E030686F
S31508008310406A19EA00002070641C07E0002CF6D1B8
S315080083203068406A19EA00002880AD1CB6F85A0081
S31508008330401EA6F85A00B6F85A0000280AD0009738
S31508008340434600222021300000F064FA0028E5D0D8
S31508008350032007E02020B067002086F87000002080
S3150800836000E00220BDE8F28338B5040000210025AC
S31508008370A2682069024360690243E06902432068F3
S315080083800368DFF8440303401A4320680260206844
S31508008390426832F44052E068024320684260A269AB
S315080083A0206A02432068806830F4306002432068FF
S315080083B082602068DFF81423904216D1DFF8100394
S315080083C0006810F00300002805D0022805D006D35F
S315080083D0032806D007E00120D3E00220D1E00420DC
S315080083E0CFE00820CDE01020CBE02068DFF8E422BB
S315080083F0904217D1DFF8D802006810F00C00002868
S3150800840006D0042808D0082804D00C2806D007E08F
S315080084100020B6E00220B4E00420B2E00820B0E074
S315080084201020AEE02068AC4A904216D1A8480068F1
S3150800843010F03000002806D0102808D0202804D0D4
S31508008440302806D007E000209BE0022099E00420AF
S3150800845097E0082095E0102093E020689F4A904214
S3150800846016D19B48006810F0C000002806D04028A6
S3150800847008D0802804D0C02806D007E0002080E075
S3150800848002207EE004207CE008207AE0102078E0D4
S315080084902068934A904219D18D48006810F44070BC
S315080084A0002809D0B0F5807F0AD0B0F5007F05D046
S315080084B0B0F5407F06D007E0002062E0022060E0C9
S315080084C004205EE008205CE010205AE02068854A17
S315080084D0904219D17E48006810F44060002809D0FF
S315080084E0B0F5806F0AD0B0F5006F05D0B0F5406FD3
S315080084F006D007E0012044E0022042E0042040E0E4
S3150800850008203EE010203CE02068774A904219D1C6
S315080085106F48006810F44050002809D0B0F5805F15
S315080085200AD0B0F5005F05D0B0F5405F06D007E089
S31508008530002026E0022024E0042022E0082020E093
S3150800854010201EE02068694A904219D160480068E8
S3150800855010F44040002809D0B0F5804F0AD0B0F595
S31508008560004F05D0B0F5404F06D007E0002008E0E0
S31508008570022006E0042004E0082002E0102000E0C3
S315080085801020E269B2F5004F4FD1C0B2002808D0DA
S31508008590012811D002281AD0042821D008282AD068
S315080085A032E000F031FC6168490811EB400160686F
S315080085B0B1FBF0F189B228E000F031FC61684908A6
S315080085C011EB40016068B1FBF0F189B21DE060680B
S315080085D0474911EB50016068B1FBF0F189B214E02C
S315080085E000F0D7FB6168490811EB40016068B1FBF0
S315080085F0F0F189B209E06068400810F580306168DA
S31508008600B0FBF1F189B200E001254FF6F072B1F145
S315080086101000904207D20A40C1F34200024392B2C8
S315080086202068C26048E0012546E0C0B2002808D0AC
S31508008630012810D0022818D004281FD0082827D0CF
S315080086402FE000F0E1FB616810EB51006168B0FBB8
S31508008650F1F189B226E000F0E2FB616810EB510007
S315080086606168B0FBF1F189B21CE06068214911EB41
S3150800867050016068B1FBF0F189B213E000F089FBA4
S31508008680616810EB51006168B0FBF1F189B209E04D
S315080086906068400810F500406168B0FBF1F189B2E6
S315080086A000E00125B1F110004FF6F072904202D2B7
S315080086B02068C16000E00125002020660020606671
S315080086C02800C0B232BD0000F369FFEF0010014078
S315080086D0903802400044004000480040004C0040EA
S315080086E0005000400014014000780040007C004023
S315080086F00048E8010024F40090F82410C90707D5BB
S3150800870001684A6832F40032816A0A4301684A609D
S3150800871090F82410890707D501684A6832F4803230
S31508008720C16A0A4301684A6090F82410490707D5C8
S3150800873001684A6832F48022016B0A4301684A607C
S3150800874090F82410090707D501684A6832F40042F0
S31508008750416B0A4301684A6090F82410C90607D598
S3150800876001688A6832F48052816B0A4301688A601C
S3150800877090F82410890607D501688A6832F40052F1
S31508008780C16B0A4301688A6090F82410490613D51C
S3150800879001684A6832F48012016C0A4301684A602B
S315080087A0016CB1F5801F07D101684A6832F4C0022E
S315080087B0416C0A4301684A6090F82410090607D5F7
S315080087C001684A6832F40022816C0A4300684260F4
S315080087D070471CB504000020E06700F051F803005C
S315080087E02068006800070CD57FF07E4000900022C4
S315080087F05FF40011200000F00DF8002801D00320D6
S3150800880007E0202060672020A067002084F8700019
S31508008810002016BD2DE9F04105000E0090461F0008
S31508008820069C2868C0693040B04201D1012000E0AA
S3150800883000204146C9B288421ED114F1010FF0D07A
S3150800884000F01EF8C01B844201D3002CE9D1286829
S31508008850006830F4D0702968086028688068400885
S31508008860400029688860202068672020A8670020C3
S3150800887085F87000032000E00020BDE8F08170470D
S3150800888001480068704700BF000100202DE9FC413F
S3150800889004000025002C01D10120D1E12078C00771
S315080088A06DD5DFF89405016811F00C01042909D08B
S315080088B0006810F00C0008280ED1DFF88005006863
S315080088C0400209D5DFF86C050068800357D5606853
S315080088D0002854D10120B3E16068B0F5803F06D185
S315080088E0DFF85005016851F48031016026E06068C0
S315080088F000280AD1DFF83C05016831F480310160AF
S31508008900016831F48021016018E06068B0F5A02F95
S315080089100AD1DFF82005016851F480210160016859
S3150800892051F48031016009E0DFF80805016831F487
S3150800893080310160016831F4802101606068002897
S315080089400ED0FFF79DFF0600DFF8E80400688003F5
S3150800895015D4FFF795FF801B6528F5D303206FE133
S31508008960FFF78EFF0600DFF8CC040068800306D503
S31508008970FFF786FF801B6528F5D3032060E1207882
S31508008980800720D5DFF8B004016811F00C0F09D074
S31508008990006810F00C0008282ED1DFF8A004006843
S315080089A0400229D4DFF88C040168890704D5E168F8
S315080089B0012901D0012043E1016831F0F80122695B
S315080089C051EAC20101602078000759D5606900287C
S315080089D043D0DFF86C74386850F001003860FFF750
S315080089E04FFF0600386880074AD4FFF749FF801B07
S315080089F00328F7D3032023E1E06800281AD0DFF81C
S31508008A003464306850F001003060FFF739FF070022
S31508008A103068800706D4FFF733FFC01B0328F7D357
S31508008A2003200DE1306830F0F800216950EAC100F2
S31508008A303060C8E7DFF8FC733868400840003860E3
S31508008A40FFF71EFF060038688007BCD5FFF718FF3A
S31508008A50801B0328F7D30320F2E0DFF8E4733868B5
S31508008A60400840003860FFF70BFF060038688007AB
S31508008A7006D5FFF705FF801B0328F7D30320DFE0A1
S31508008A802078400740F18280DFF8C0633068C00074
S31508008A9009D4306850F080503060306810F080504B
S31508008AA0009000980125DFF8A8733868C00511D42E
S31508008AB0386850F480703860FFF7E2FE8046386800
S31508008AC0C00507D4FFF7DCFEB0EB08006528F6D32F
S31508008AD00320B5E0A068012806D1DFF8780301680D
S31508008AE051F00101016025E0A06800280AD1DFF8ED
S31508008AF064030168490849000160016831F004010E
S31508008B00016017E0A06805280AD1DFF84803016864
S31508008B1051F004010160016851F00101016009E0AA
S31508008B20DFF830030168490849000160016831F03F
S31508008B3004010160A068002810D0FFF7A1FE070015
S31508008B40DFF810030068800719D4FFF799FEC01BE9
S31508008B5041F289318842F3D3032071E0FFF790FE92
S31508008B600700DFF8F0020068800708D5FFF788FEDF
S31508008B70C01B41F289318842F3D3032060E0EDB28D
S31508008B80012D03D1306830F080503060A06900288C
S31508008B9055D0DFF8A402006810F00C0008284CD065
S31508008BA0A069022836D1DFF88C52286830F0807028
S31508008BB02860FFF765FE06002868800106D5FFF7DE
S31508008BC05FFE801B0328F7D3032039E0E169206A9A
S31508008BD00143606A51EA8011A06A4008401E51EAC2
S31508008BE00041E06A51EA006151F00051DFF84C0299
S31508008BF00160286850F080702860FFF741FE040085
S31508008C00286880011BD4FFF73BFE001B0328F7D317
S31508008C10032015E0DFF81C52286830F080702860C1
S31508008C20FFF72EFE04002868800108D5FFF728FE06
S31508008C30001B0328F7D3032002E0012000E00020F0
S31508008C40BDE8F6812DE9F04104000D000020002C56
S31508008C5001D101209BE0DFF80062306810F00F00B8
S31508008C60A8420BD2306800090001284330603068FA
S31508008C7010F00F00A84201D0012088E02078800774
S31508008C8019D52078400705D5DFF8AC01016851F4FD
S31508008C90E05101602078000705D5DFF89C010168DE
S31508008CA051F460410160DFF890110A6832F0F00271
S31508008CB0A06802430A602078C00733D56068012897
S31508008CC006D1DFF870010068800310D401205EE049
S31508008CD06068022805D157480068800107D401203A
S31508008CE055E054480068800701D401204FE0524FF0
S31508008CF0396889088900606801433960FFF7C0FD53
S31508008D008046386810F00C006168B0EB810F09D016
S31508008D10FFF7B6FDB0EB080041F289318842F0D37F
S31508008D20032034E0306810F00F0085420BD230681B
S31508008D300009000128433060306810F00F00A8428F
S31508008D4001D0012023E02078400706D53A490A6871
S31508008D5032F4E052E06802430A602078000707D53B
S31508008D603548016831F46041226951EAC20101605F
S31508008D7000F00FF83949304A1268C2F30312895CC9
S31508008D80C84031490860002000F06EF80020BDE8B0
S31508008D90F08110B500200020002000202648006839
S31508008DA010F00C00002804D0042804D0082804D0A9
S31508008DB025E0244824E02A4822E0204C226812F0C4
S31508008DC03F022068400209D52068C0F3881024496C
S31508008DD0A1FB0001002300F06DF808E02068C0F34D
S31508008DE088101849A1FB0001002300F063F82168E8
S31508008DF0C1F30141491C4900B0FBF1F000E01148FC
S31508008E0010BD11480068704780B5FFF7FAFF15498D
S31508008E10094A1268C2F38222895CC84002BD80B53D
S31508008E20FFF7EFFF0F49044A1268C2F34232895C22
S31508008E30C84002BD003802400838024004380240E3
S31508008E40743802400024F400040000204038024030
S31508008E500070004070380240003C024044A10008FF
S31508008E6000127A006CA1000810B504004FF47A705D
S31508008E700D490978B0FBF1F00C490968B1FBF0F02F
S31508008E8000F09EF9002801D001200CE0102C09D230
S31508008E90002221005FF0FF3000F081F904480460E9
S31508008EA0002000E0012010BD08000020040000207A
S31508008EB000000020BBBBE1B1B2F5803F80F07E80A8
S31508008EC0022A1ED98C46B1FBF2F102FB11C31B0420
S31508008ED043EA1043B3FBF2FC02FB1C3380B240EAC0
S31508008EE00343B3FBF2F002FB103240EA0C400023C6
S31508008EF07047022A05D98446B0FBF2F002FB10C27D
S31508008F0070474AB105D100F0010249085FEA30000E
S31508008F10704700220023704700F096B90B00020044
S31508008F20002100207047904271EB030CF6D3B3F58D
S31508008F30803F2FD2F0B5B3FA83F7B1FA81F4A7F1DF
S31508008F400F0E3D1B5340CEF1200602FA0EF2F341F6
S31508008F505340B5F10F0746D80F3C2C444140C4F1A5
S31508008F602006A040F1414140B1FBF3F603FB161180
S31508008F70A2FB0645001BA94102D2761E801859415C
S31508008F8080EA010221FA0EF362FA0EF200215A4033
S31508008F903046F0BD30B4B1FBF3FC03FB1C11A2FB59
S31508008FA00C45001BA94103D2ACF1010C80185941AC
S31508008FB030BC02460B46604600217047B2F1807FFE
S31508008FC065D3F0B5B2FA82F7B1FA81F4C7F10F06A4
S31508008FD03D1B22FA06F307F1110EF24120355A40DD
S31508008FE0B5F10F07B8D94140C4F12006A040F141B8
S31508008FF04140B1FBF3FC03FB1C11A2FB0C45001B13
S31508009000A94103D2BCF1010C801859410F2F12D384
S315080090100F3FC90341EA5041B1FBF3F603FB1611B2
S31508009020A2FB0645D4EBC030A94102D2761E8018B1
S31508009030594146EACC3C07B34140C7F12006B8403F
S31508009040F1414140B1FBF3F603FB1611A2FB0645BD
S31508009050001BA94102D2761E8018594180EA0102F6
S3150800906021FA0EF3C7F1200462FA0EF20CFA07F0A1
S315080090705A402CFA04F13043F0BD80EA010221FA85
S315080090800EF3002162FA0EF260465A40F0BD8C4695
S31508009090B1FBF2F102FB11C31B0243EA1063B3FBF7
S315080090A0F2FC02FB1C331B024CEA002043EA106365
S315080090B0B3FBF2FC02FB1C331B024CEA002043EA1A
S315080090C01063B3FBF2FC02FB1C331B024CEA0020C4
S315080090D043EA1063B3FBF2FC02FB1C324CEA0020A5
S315080090E00023704710F007003F4B1A684FF6FF0140
S315080090F00A403E4951EA00210A431A6070473A4835
S315080091000068C0F302207047020052B2002A04D455
S315080091100901374A40B2115407E00901354A40B2FD
S3150800912010F00F00104400F8041C704710B410F03B
S315080091300700D0F10703052B01D3042301E0D0F182
S315080091400703041D072C01D2002000E0C01E0124DD
S3150800915014FA03F35B1E1940814014FA00F0401E0E
S315080091601040084310BC704780B5411EB1F1807F9E
S3150800917001D301200EE0401E1F4908600F215FF051
S31508009180FF30FFF7C1FF00201C49086007201C4973
S315080091900860002002BD80B5FFF7A4FF01BD70B5C9
S315080091A004000D0016000020FFF7A9FF3200290071
S315080091B0FFF7BCFF0100200040B2FFF7A5FF70BD16
S315080091C080B5FFF7D1FF02BD042805D10C48016818
S315080091D051F00401016004E00948016831F0040116
S315080091E001607047000000000CED00E00000FA0581
S315080091F000E400E018ED00E014E000E018E000E00C
S3150800920010E000E080B500F001F801BD704730B409
S31508009210002513E050F8042BD30744BFA9F1010336
S315080092209A18091F042942F8045BFAD213468C07D8
S3150800923044BF15809B1CC90748BF1D7050F8041B06
S315080092400029E7D130BC7047704730B40EE0026899
S31508009250436802440830DC0744BFA9F10104E31857
S3150800926052F8045B43F8045B091FF9D150F8041B54
S315080092700029ECD130BC704738B50400002C01D168
S315080092800120AEE094F82000002802D1200000F06A
S3150800929015FA2068006830F0020021680860FFF7B8
S315080092A0EFFA05002068406880070DD5FFF7E8FA51
S315080092B0401B0B28F6D3606A50F400306062052024
S315080092C084F8200001208CE02068006850F0010036
S315080092D021680860FFF7D4FA050020684068C007CF
S315080092E00DD4FFF7CDFA401B0B28F6D3606A50F46D
S315080092F000306062052084F82000012071E0207E9D
S31508009300012806D12068006850F0800021680860AE
S3150800931005E02068006830F0800021680860607EFB
S31508009320012806D12068006850F0400021680860CE
S3150800933005E02068006830F0400021680860A07EDB
S31508009340012806D12068006850F0200021680860CE
S3150800935005E02068006830F0200021680860E07E9B
S31508009360012806D12068006830F0100021680860DE
S3150800937005E02068006850F0100021680860207F2A
S31508009380012806D12068006850F0080021680860A6
S3150800939005E02068006830F0080021680860607FF2
S315080093A0012806D12068006850F00400216808608A
S315080093B005E02068006830F0040021680860A168AC
S315080093C0E068014320690143606901436068401E03
S315080093D001432068C16100206062012084F82000F2
S315080093E0002032BD30B4026890F820201300DBB2AA
S315080093F0012B03D0D2B2022A40F07F80594AD2F814
S31508009400000250F00100C2F80002D2F8000230F45F
S315080094107C50C2F80002D2F800024B6A50EA0320D8
S31508009420C2F8000201200B7D13F01F0310FA03F3A4
S31508009430D2F81C029843C2F81C02C869002816D143
S31508009440D2F80C029843C2F80C02486902EBC00035
S31508009450CC684D68C5EA0444C0F84042486902EB46
S31508009460C0008C680D68C5EA0444C0F84442C8695F
S31508009470012816D1D2F80C021843C2F80C02486922
S3150800948002EBC0000C684D68C5EA0444C0F84042C7
S31508009490486902EBC0008C68CD68C5EA0444C0F888
S315080094A044428869002805D1D2F804029843C2F8D4
S315080094B0040204E0D2F804021843C2F80402086958
S315080094C0002805D1D2F814029843C2F8140204E021
S315080094D0D2F814021843C2F81402086A012804D103
S315080094E0D2F81C020343C2F81C32D2F80002400824
S315080094F04000C2F80002002004E0416A51F48021CD
S315080095004162012030BC704738B5040094F8200049
S31508009510012821D1022084F820002068006840082C
S31508009520400021680860FFF7ABF90500206840682D
S31508009530C0070DD5FFF7A4F9401B0B28F6D3606AC0
S3150800954050F400306062052084F82000012008E00D
S3150800955000206062002004E0606A50F40020606227
S31508009560012032BD0064004030B490F82040250048
S31508009570EDB2012D03D0E4B2022C40F09880002908
S315080095800AD10468E46814F0030F10D1416A51F453
S315080095900011416201208FE00468246914F0030F6A
S315080095A005D1416A51F400114162012084E0046842
S315080095B00D012C44D4F8B04114F004049460946866
S315080095C0002C07D104680D012C44D4F8B041640D71
S315080095D0146006E004680D012C44D4F8B041E40890
S315080095E0546004680D012C44D4F8B041C4F3400417
S315080095F0D46004680D012C44D4F8B44114F00F0467
S31508009600146104680D012C44D4F8B441C4F307244A
S31508009610946104680D012C44D4F8B441240C5461B7
S3150800962002680C012244D2F8B8211A7002680C01AB
S315080096302244D2F8B821120A5A7002680C01224450
S31508009640D2F8B821120C9A7002680C012244D2F89A
S31508009650B821120EDA7002680C012244D2F8BC2135
S315080096601A7102680C012244D2F8BC21120A5A71F6
S3150800967002680C012244D2F8BC21120C9A710268C5
S315080096800C012244D2F8BC21120EDA71002906D147
S315080096900168C96851F020010068C16005E00168E9
S315080096A0096951F0200100680161002004E0416A5F
S315080096B051F480214162012030BC70477047000098
S315080096C0BFF34F8FB6490A6812F4E062B548024301
S315080096D00A60BFF34F8F00BFFDE780B500F00DF8B5
S315080096E000F0CDF801BD80B500F021F800F02AF9A8
S315080096F001BD80B5FFF7E4FF01BD80B5AA48AB49B7
S3150800970001604FF461414160002181600021C16020
S31508009710002101610C214161002181610021C161A3
S315080097200021016200214162FEF750FD01BD70B5BE
S315080097309F4C2078002815D19E4D280000F037F858
S31508009740012833D12878002830D0287841282DDA06
S3150800975000F053F9984908600120207000209749C5
S31508009760087023E0954D934E28783044401C00F04D
S315080097701EF8012811D12878401C287028783178DD
S31508009780884213D1002020707078FF280ED12878DF
S3150800979002280BD1FFF7ADFF08E000F02EF9864945
S315080097A009686431814201D20020207070BD80B5FD
S315080097B00100002301227C48FEF745FDC0B20028BF
S315080097C001D1012000E0002002BDF8B504000D001B
S315080097D016001F00FFF718FB4FF47A71B0FBF1F182
S315080097E0002200E0521C1000C0B2122845D2744B69
S315080097F0200080B294465FFA8CFC13F81CC096468B
S315080098005FFA8EFE03EB4E0E9EF801E01EEB0C0C83
S315080098101CF1010C0CFB00F0B1FBF0FC00FB1C106A
S315080098200028DFD1200080B294465FFA8CFC13F83A
S315080098301CC096465FFA8EFE03EB4E0E9EF801E0BC
S315080098401EEB0C0C1CF1010C0CFB00F0B1FBF0F04C
S31508009850288028880028C5D0288840F2014C604511
S31508009860C0DA1000C0B213F810003070D2B203EBA1
S31508009870420040783870012000E00020F2BD30B583
S315080098808BB00020ADF8020000208DF80100002002
S315080098908DF8000040F267656B460DF101020DF187
S315080098A002014FF4FA70FFF790FF464C46482060D5
S315080098B000202076002060760020A0760120E07641
S315080098C000202077002060770020A0600020E0605C
S315080098D09DF80100401E000420619DF80000401E0E
S315080098E000056061BDF8020060602000FFF7C4FC57
S315080098F0002D02D46D05354805E025F00045ED003C
S3150800990055F00405324800210691002107910121EE
S3150800991008912900090C0191ADB202950100090CC4
S31508009920039180B2049000200590012009900E2032
S315080099300A9001A92000FFF755FD2000FFF7E4FD76
S315080099400BB030BD30B589B040F2676400256B4670
S3150800995002AA00211B48FFF707FE00281ED1002C8B
S3150800996007D40298A0420DD1049800280AD10125EF
S3150800997008E024F000440398A04203D10498042880
S3150800998000D10125EDB2012D08D19DF80000FF2870
S3150800999004D10698022801D1FFF7ABFE09B030BD05
S315080099A00CED00E00400FA050C0000200048004019
S315080099B0050100208C000020F8000020040100208A
S315080099C078A00008D0000020006400400400E0FFF2
S315080099D0FCFF1F0080B5FFF714FA4FF47A71B0FB4D
S315080099E0F1F0FFF7EDFB0420FFF7EEFB0022002164
S315080099F05FF0FF30FFF7D3FB01BD80B5FEF740FFF0
S31508009A0002BD80B500F004F8FFF7FCFB01BD0000BD
S31508009A1003480168034A127889180160704700BF35
S31508009A200001002008000020F8B4002200220022CD
S31508009A300022002337E00A2704E0DFF8F0219042ED
S31508009A40F9D10927FFB213F00302D2B29200974068
S31508009A503E431A00920845F82260DFF8D4512A6876
S31508009A60A2434E68F60300D522432A60DFF8C451A4
S31508009A702A68A2434E68B60300D522432A60DFF857
S31508009A80B8512A68A2434E68F60200D522432A60D6
S31508009A90DFF8A8512A68A2434E68B60201D51443D6
S31508009AA022002A605B1C102B80F0B380012515FA72
S31508009AB003F20C6814409442F4D14A68022A02D090
S31508009AC04A68122A17D11A00D20800EB8202166ACF
S31508009AD00F2713F00702D2B292009740BE430F69D0
S31508009AE013F00702D2B2920097403E431A00D208FA
S31508009AF000EB82021662076803261A00D2B25200E9
S31508009B0016FA02F2974391F804C01CF0030C1A00E7
S31508009B10D2B252001CFA02FC5CEA070707604A68E0
S31508009B20012A08D04A68022A05D04A68112A02D0B2
S31508009B304A68122A19D187681A00D2B2520016FA50
S31508009B4002F29743D1F80CC01A00D2B252001CFA9E
S31508009B5002FC5CEA0707876042689D40AA434D6895
S31508009B60C5F300159D402A434260C5681A00D2B263
S31508009B7052009640B5438E681A00D2B252009640FB
S31508009B803543C5604A68D2008CD52D4A156855F408
S31508009B9080451560126812F480420092009A294D99
S31508009BA01A00920855F822600F2713F00302D2B262
S31508009BB092009740BE43244A904201D1002741E7CC
S31508009BC0224A904201D101273CE7214A904201D11D
S31508009BD0022737E71F4A904201D1032732E71E4A78
S31508009BE0904201D104272DE71C4A904201D105274E
S31508009BF028E71B4A904201D1062723E7194A9042D3
S31508009C0001D107271EE7184A90427FF416AF0827A6
S31508009C1018E7F1BC7047D2B2002A02D089B2816136
S31508009C2002E089B2090481617047000000240240FD
S31508009C30003C0140043C0140083C01400C3C01400A
S31508009C40443802400838014000000240000402403F
S31508009C5000080240000C02400010024000140240B6
S31508009C6000180240001C02400020024080B500F0A7
S31508009C7007F8FFF732FD00F010F9FFF734FDFAE7B1
S31508009C8080B500F009F800F02DF900F009F8FFF7A3
S31508009C90A1FE00F0FBF801BD7448754908607047DD
S31508009CA080B592B03022002106A800F026F91422C9
S31508009CB0002101A800F021F96E48016851F0805191
S31508009CC00160006810F08050009000986A480168AA
S31508009CD051F440410160006810F44040009000983B
S31508009CE0012006905FF4A020079002200C905FF4F4
S31508009CF080000D9008200E904FF4D8700F90022027
S31508009D0010900220119006A8FEF7C0FD002800D08A
S31508009D10FEE700F0FDF8002800D0FEE70F200190CE
S31508009D2002200290002003904FF4A05004904FF4B4
S31508009D3080500590072101A8FEF784FF002800D06F
S31508009D40FEE713B000BD38B586B04A48016851F041
S31508009D5080510160016811F08051059105994749C4
S31508009D600A6852F480420A60096811F48041059134
S31508009D70059943490A6852F002020A600A6812F015
S31508009D8002020592059A0A6852F008020A600968F2
S31508009D9011F0080105910599016851F480210160C7
S31508009DA0016811F4802105910599016851F0007147
S31508009DB00160006810F00070059005980320FFF711
S31508009DC0EAF9002200217FF00B00FFF7E8F90022EC
S31508009DD000217FF00A00FFF7E2F9002200217FF058
S31508009DE00900FFF7DCF9002200217FF00400FFF7E5
S31508009DF0D6F9002200217FF00300FFF7D0F90022F0
S31508009E0000217FF00100FFF7CAF9002200215FF068
S31508009E10FF30FFF7C4F98020009001200190002050
S31508009E20029000200390174C69462000FFF7FCFDBE
S31508009E304FF44075009502200190002002900320FF
S31508009E4003900720049069460F48FFF7EDFD00953B
S31508009E50022001900020029003200390092004901C
S31508009E6069462000FFF7E0FD07B030BD0080000816
S31508009E7008ED00E0403802400070004044380240D7
S31508009E803038024000040240000C024080B500222F
S31508009E9080211148FFF7BFFE01BD38B5FFF7ADFDBC
S31508009EA004000E4D2868201AB0F5FA7F13D30C4922
S31508009EB00878002807D10120087001228021064869
S31508009EC0FFF7A9FE06E0002008700022802102485C
S31508009ED0FFF7A1FE2C6031BD00040240FC00002003
S31508009EE00601002080B50320FFF755F90020FEF78C
S31508009EF0BBFFFFF728FF002002BD10B50446104639
S31508009F000A460146204600F03FF8204610BD0000EC
S31508009F107CB500201B48016851F08051016000683B
S31508009F2010F0805000900098154E306850F480303C
S31508009F303060FEF7A5FC0500104C2068C00308D465
S31508009F40FEF79EFC401B40F2E9318842F4D3032019
S31508009F5013E0306850F400303060FEF791FC0500DD
S31508009F602068800308D4FEF78BFC401B40F2E931D9
S31508009F708842F5D3032000E0002076BD0470004037
S31508009F80007000404038024062F30F2262F31F421D
S31508009F90401810F0030308D0C91A1FD3DB0748BFBF
S31508009FA000F8012D28BF20F8022D130030B41446FE
S31508009FB01546103928BF20E93C00FAD8490728BFBA
S31508009FC020E90C0048BF40F8042D890028BF20F876
S31508009FD0022D48BF00F8012D30BC7047C91818BFBC
S31508009FE000F8012DCB0728BF00F8012D70470000A7
S31508009FF00F48016851F4700101600E49086850F075
S3150800A0000100086000200C4A10600A680B480240EC
S3150800A0100A600B480B4A1060086830F48020086014
S3150800A0200020094908605FF0006008490860704729
S3150800A03088ED00E00038024008380240FFFFF6FECF
S3150800A04010300024043802400C38024008ED00E0C5
S3150800A05010B5074979441831064C7C44163404E097
S3150800A0600A68081D114488470146A142F8D110BD67
S3150800A07050000000700000000502060206030703F0
S3150800A0800803090309040A040B040C040C050D054E
S3150800A0900E050F050F061006100710084EF6885114
S3150800A0A0CEF20001086840F470000860BFF34F8FD5
S3150800A0B0BFF36F8F4FF00070E1EE100A7047000093
S3150800A0C04FF1FFFFFC0000000C000020000000001C
S3150800A0D07BF1FFFF0C000000880000000000002054
S3150800A0E00000000000F00DF8002801D0FFF7B0FFCF
S3150800A0F0AFF300800020AFF30080FFF7B7FD00F054
S3150800A10002F80120704700F001B8000007463846FB
S3150800A11000F002F8FBE7000080B5AFF30080024AC2
S3150800A12011001820ABBEFBE7260002000248854650
S3150800A130024880470248004708050020F19F0008AA
S3150800A14055A10008000000000000000001020304F9
S3150800A15006070809AFF30080FFF7A0FFFFF7C2FF65
S3150800A160100000000024F4000100000000000000B8
S3150800A17001020304FFF7FEBFFFF7FEBFFFF7FEBFAE
S3150800A180FFF7FEBFFFF7FEBFFFF7FEBFFFF7FEBFF5
S3150800A190FFF7FEBFFFF7FEBFFFF7FEBFFFF7FEBFE5
S3150800A1A0FFF7FEBFFFF7FEBFFFF7FEBFFFF7FEBFD5
S3150800A1B0FFF7FEBFFFF7FEBFFFF7FEBFFFF7FEBFC5
S3150800A1C0FFF7FEBFFFF7FEBFFFF7FEBFFFF7FEBFB5
S3150800A1D0FFF7FEBFFFF7FEBFFFF7FEBFFFF7FEBFA5
S3150800A1E0FFF7FEBFFFF7FEBFFFF7FEBFFFF7FEBF95
S3150800A1F0FFF7FEBFFFF7FEBFFFF7FEBFFFF7FEBF85
S3150800A200FFF7FEBFFFF7FEBFFFF7FEBFFFF7FEBF74
S3150800A210FFF7FEBFFFF7FEBFFFF7FEBFFFF7FEBF64
S3150800A220FFF7FEBFFFF7FEBFFFF7FEBFFFF7FEBF54
S3150800A230FFF7FEBFFFF7FEBFFFF7FEBFFFF7FEBF44
S3150800A240FFF7FEBFFFF7FEBFFFF7FEBFFFF7FEBF34
S3150800A250FFF7FEBFFFF7FEBFFFF7FEBFFFF7FEBF24
S3150800A260FFF7FEBFFFF7FEBFFFF7FEBFFFF7FEBF14
S3150800A270FFF7FEBFFFF7FEBFFFF7FEBFFFF7FEBF04
S3150800A280FFF7FEBFFFF7FEBFFFF7FEBFFFF7FEBFF4
S3150800A290FFF7FEBFFFF7FEBFFFF7FEBFFFF7FEBFE4
S3150800A2A0FFF7FEBFFFF7FEBFFFF7FEBFFFF7FEBFD4
S3150800A2B0FFF7FEBFFFF7FEBFFFF7FEBFFFF7FEBFC4
S3150800A2C0FFF7FEBFFFF7FEBFFFF7FEBFFFF7FEBFB4
S3150800A2D0FFF7FEBFFFF7FEBFFFF7FEBFFFF7FEBFA4
S3150800A2E0FFF7FEBFFFF7FEBFFFF7FEBFFFF7FEBF94
S3150800A2F0FFF7FEBFFFF7FEBFFFF7FEBFFFF7FEBF84
S3150800A300FFF7FEBFFFF7FEBFFFF7FEBFFFF7FEBF73
S30D0800A310FFF7FEBFFFF7FEBFD1
S7050800A155FC
